:100000002500DA0C0600C00C0200A405A305320A84
:10001000A404A3042200E2013008010800080B0830
:10002000010800080008000800080A082E083C081B
:100030009C0819087A080C08B8086608AE08F00889
:10004000DF08C008260805083D08070842084908D7
:1000500052084F084408320842080F08470872083F
:1000600061086D086C08690863086808260842087A
:1000700065086E0873086F086E08A4047705A40568
:100080008607460AA4049709A405400AA605A40405
:10009000970997099709A405720000000000000065
:1000A00000000000080C3100A40497090304A40513
:1000B00032038606F205A4049709970900000000A0
:1000C000A405F102540AA40497099709A405120291
:1000D00030000008A404430477064305A405430741
:1000E000760AA404770497099709A405A604A40432
:1000F000970997099709080CA40534001307A6046B
:100100001306A60503043303A40497099709970966
:10011000A405F4027E0A0000A605A4049709970925
:1001200097090000000000000000A405000804007A
:10013000F20043070D0B080C3200B302D300430654
:10014000DD0A330C93004306BB0A340C93004306CC
:10015000B00A000000000000000000000000B70A24
:10016000030C670108070704280727047300000031
:1001700000000000D90A0607C20A000000000000C3
:100180000000CA0A960426079605960707049606F5
:10019000070506054607D10A000000000000000020
:1001A000D90A96046607960596072704960627053A
:1001B0004605000000000000080BB4020806E60A2D
:1001C00000000000000000000000F30A5707EF0ADB
:1001D0005706EC0A0000EE0A14060604F30A0000B3
:1001E00000000000ED0A2806FB0A000000000000E5
:1001F00000000000080B5707040B5706010B000016
:10020000030B14074604080B000000000000020B5B
:100210000000000000000000360B0F023000070253
:100220008901030E2F00030C8F0131000F02900192
:100230002E000C02510135000B024F0135010E0258
:100240004F014D0135010E0250014A0115014307CE
:10025000370537062E0B00000000360B1707330B4F
:10026000A6041704360B0000000000001D0C35002A
:08027000F502380B0000000844
:10040000E201570A5F0A650A740A7E0A880A920A9C
:10041000920AE201540A9D0A9E0A9E0AA70AA70AA6
:10042000B00AB00AE201E30AE30AE30AE30AF60AC1
:10043000F60A010B010BE2010F0B120B150B1B0B44
:10044000200B320B340B3B0BE2013E0B3E0B3E0B01
:100450003E0B3E0BC00AE00A0C0BE2014E0AB90A41
:10046000B90ABA0AA60506054605A4041704370406
:100470005704030C280069006A006B006C006D00D3
:10048000A40576007700A3043D091002350095030A
:10049000390039031903030EA3052D0A150339008A
:1004A000390319031F0E090A070C5501000A070238
:1004B00089010F0E3300A3046A09A3059C0A0702F1
:1004C0003300A3046A09A3059C0AA4044304570645
:1004D0004305A40543066E0A7300700A010C33003D
:1004E000A3046A09A3059C0A480339005903FC0EBA
:1004F00009013300A3046A09A3059C0A4B033900D0
:100500005903FC0E0C013300A3046A09A3059C0ADD
:100510004D0339005903FC0E0A013300A3046A0994
:10052000A3059C0AA4045704A40543041506430527
:10053000A40443065705A405B80AB80A15033900F0
:100540001903030E2800030C55012900B80A1503EE
:1005500039001903030E2B00030C55012C00B80AB7
:10056000150339001903030E2D00030C55012A0051
:100570003E0B3E0B1503390039031903070E240AFD
:10058000070C55013900070C99004307DF0A780072
:10059000A404430417064305A4054307D10A020C2B
:1005A0003801A404430437064305A4054307DA0AC7
:1005B000010C380118023300A3046A09A3053E0B9D
:1005C000070C5501120AA4041704A40543043506B8
:1005D0004305A404430617053704A4054304150680
:1005E0004305A40443063705A4050B0BA4043704F4
:1005F000A405430415064305A40443063705A405D2
:100600000B0BA4041704A405430415064305A40416
:1006100043061705A4053E0B070C55011B0AFC0CED
:10062000E5013E0B040CE5013E0B05023300A3047B
:100630006A09A3053E0B7300A3046A09A3053E0BD8
:10064000300C9700030677009702A404A3040B095B
:10065000A40533006A09B702300C9700A30503060E
:1006600077003E0B77003E0B16023300A3046A09A5
:0E0670007600A3053E0B96024307B602430A2E
:021FFE000E00D3
:00000001FF
